:10000000E0EF04F000000000C2EF04F00000000088
:0A0010000000000000000000F3D71C
:10001C00026A036A800E0318006E800E005C02E117
:10002C00080E025C11E28296800E01017515016EBC
:10003C000150800A02E1828801D08298828675374D
:0A004C007591024A032AE6D712005C
:0E0056008282829074C175F1DEDF828012001A
:100064008292829074C175F1D7DF070E0C6E7D0EFB
:0E0074000D6E0D2EFED70C2EFCD782801200D2
:0600820000000000120066
:100088000FEE81F0EF50EFCF00F0009E00C0EFFFC1
:02009800120054
:10009A000FEE81F0EF50EFCF00F0009C00C0EFFFB1
:0200AA00120042
:1000AC006FC102F070C103F002C000F003C001F098
:1000BC00024A032A00C0E9FF01C0EAFFEE5201E048
:1000CC00F3D701016F51025C006E70510358016E41
:0A00DC00010E005E000E015A120032
:1000E600070E01017015006E400E0010746FB7DF29
:1000F6007F0E01016F15006E800E0010746FAFDF6A
:020106001200E5
:10010800200E01016F5D04E36F517F0801E301D008
:100118001200050E6F03F3CF00F0F4CF01F0A00E2C
:10012800005C706F000E0158716F050E726F000E43
:10013800736F800E006E800E7319005C02E17251BD
:10014800000818E2DA0E7025F66E0F0E7121F76EB0
:10015800000EF86E000E71BFFF0EF8220900F5CFF1
:1001680074F175DF0101704B712B010E725F000E87
:0A017800735BDFD7746B6BDF1200BE
:0E018200ACB202D00000FCD76FC1ADFF12007E
:0A019000120E0D6E0D2EFED71200A8
:10019A00086A096A100E0C6E0134083609360450D2
:1001AA00085E0550D8A0053C095ED8B007D00450B7
:1001BA0008260550D8B0053C0926D89000360136E5
:0601CA000C2EEAD7120022
:1001D000938C57DF56DF938E54DF53DF5EDF939CA3
:0A01E00050DF4FDF51DF939E120045
:1001EA0001016C6B050E6C5D0AE26C516A25E16EC9
:1001FA00000E6B21E26E200EE66E6C2BF3D76C516B
:10020A006A25E16E000E6B21E26EE66A6C076C519C
:10021A006A256D6F000E6B216E6F0A0E046E000E5A
:10022A00056E68C100F069C101F0B2DF08C000F0D4
:10023A0009C001F0300E00266DC1E1FF6EC1E2FF78
:10024A0000C0E6FF0A0E046E000E056E68C100F0DB
:10025A0069C101F09DDF00C068F101C069F1000EBB
:10026A00011802E1000E001801E102D06C07CFD795
:02027A00120070
:10027C0001016F6B706B31DF0101686B696B800E74
:10028C00020A006E800E6919005C02E168514C088C
:10029C0010E3746BDADE040E0C6E3D0E0D6E0D2E3B
:1002AC00FED70C2EFCD7000000000101684B692B17
:0402BC00E6D712006F
:1002C000C26AC00EC212C18CC18E68C100F0003675
:1002D000009000360090003600900050C212C2809C
:1002E00057DFC284C2A401D0FDD7C4CF01F0006A99
:0C02F000C3500012000E0112C290120058
:1002FC00CEDE939CC0DEBFDE938E0101409181BEA9
:10030C0004D040A101D001D0FAD7B5DEB4DEB3DE03
:10031C00B2DEB1DEB0DEAFDEAEDE938CACDEABDED9
:02032C001200BD
:10032E00010E0101696F000E6A6F800E6B6F000E79
:10033E006C6F6B516C1123E09DDE9CDE9BDE9ADEB2
:10034E009CDE939E97DE96DE6B516815006E000E56
:10035E006C15016E0050011002E0938C02D096DEF7
:10036E00939C88DE87DE938E409181BE04D040A19F
:10037E0001D001D0FAD76C336B336C9FDAD7696B2F
:10038E006A6B78DE77DE79DE939E74DE73DE938C95
:10039E0071DE70DE6FDE6EDE938E409181BE04D014
:1003AE0040A101D001D0FAD7696B6A6B63DE62DEC1
:1003BE0081AC01D069815EDE5DDE5CDE5BDE5ADE25
:1003CE0059DE58DE57DE56DE55DE54DE53DE52DE83
:1003DE0051DE50DE4FDE51DE939E58DE939C69C196
:0403EE0000F0120009
:1003F20068C104F069C105F004C0E9FF05C0EAFF65
:10040200EE5203E0044A052AF7D704C002F005C001
:1004120003F0044A052A6AC100F06BC101F0010130
:100422006A4B6B2B00C0E9FF01C0EAFF02C0E1FF8B
:1004320003C0E2FFEECFE6FF02C0E9FF03C0EAFF1E
:10044200EE5201E0E2D768C100F069C101F012008A
:1004520068C104F069C105F004C002F005C003F0F0
:10046200044A052A6AC100F06BC101F001016A4B1E
:100472006B2B00C0E9FF01C0EAFF02C0E1FF03C02D
:10048200E2FFEECFE6FF02C0E9FF03C0EAFFEE5251
:0E04920001E0E2D768C100F069C101F012007C
:1004A00003C16FF104C170F101DE00C069F1686B36
:1004B00068510325E96E000E68BFFF0E0421EA6E45
:1004C000EECF6AF154A104D06AC16FF15ADE03D0B5
:1004D0006AC16FF119DE0101682B800E6819006E88
:1004E000800E6919005CE4E319D029D028D02C0EC5
:1004F0006F6F47DE24D0090E01016F6F42DE1FD0FF
:100500000D0E01016F6F3DDE0A0E01016F6F39DEC6
:1005100016D02A0E01016F6F34DE11D00101545143
:10052000000AE3E05451010AE1E05451030ADFE01C
:100530005451050AE0E05451070AE2E0EAD71200FC
:10054000800E01016A6F000E6B6F6C6B6D6B6A51F0
:100550006B111BE096DD95DD938C93DD92DD938E20
:10056000409181BE04D040A101D001D0FAD781AC26
:1005700004D06A516C136B516D1383DD82DD84DD11
:10058000939E6B336A336B9FE2D7938C7ADD79DD70
:100590006851691102E081DD939C73DD72DD938EF9
:1005A000409181BE04D040A101D001D0FAD769DDCD
:1005B00068DD6ADD939E65DD64DD6FDD939C6CC153
:0405C00000F0120035
:1005C4000A0E01016F6FDBDD0D0E01016F6FD7DDC8
:0205D400120013
:0A05D600000E9EBA010E006E120026
:1005E000AECF3DF1ABA202D0AB98AB883DC100F0DD
:0205F0001200F7
:1005F200A6A202D00000FCD7A69C66C1A9FF67C1D3
:10060200A8FFA69EA684F2CF00F0F29E550EA76E1A
:10061200AA0EA76EA68200BE02D0F29E01D0F28E72
:04062200A694120088
:10062600A69C66C1A9FFA69EA680A8CF00F01200D0
:10063600828482808294020E0B6E450E0C6EA90E89
:100646000D6E0D2EFED70C2EFCD70B2EFAD7000002
:1006560000008284210E0101746F01DD900E0101FC
:10066600746FFDDC050E0101746FF9DC130E0101D8
:10067600746FF5DC200E0101746FF1DC210E0C6E37
:10068600760E0D6E0D2EFED70C2EFCD700000C0E2E
:100696000101746FE4DCEFDD210E0C6E760E0D6E3B
:1006A6000D2EFED70C2EFCD700006F6B706B18DD7D
:0206B600120030
:1006B8000900F5CFE6FF0006FBE10106F9E11200AB
:1006C80001015951800F586F5B5158275A515827CB
:1006D8007BDDD00E686F27DE58C168F124DE0ADEA4
:1006E800040E0C6E3D0E0D6E0D2EFED70C2EFCD793
:1006F8000000000069DDD10E0101686F14DE010EF3
:10070800686F000E696F18DF00C066F1010E686F30
:10071800000E696F11DF00C067F1686B696B0CDF51
:10072800E9DD66C101F0006A010167510026000E8B
:040738000122120088
:10073C000B6A0A6A096A00500402F4CF09F0F3CF7D
:10074C0008F001500502F4CF0BF0F3CF0AF0005083
:10075C000502F3500926F4500A22E86A0B220150D4
:10076C000402F3500926F4500A22E86A0B2208C04E
:10077C0000F009C001F00AC002F00BC003F0120037
:10078C00820E0101506F010E516F6F0E526F010EF0
:10079C00536FE00E476F050E486F000E496F000E49
:1007AC004A6FD60E4B6F050E4C6F000E4D6F000E40
:1007BC004E6FFF0E416FFF0E426F000E436F000E27
:1007CC00446FAC8A900EAB6E948E949C9EAA03D010
:0807DC00AECF00F0FBD71200C4
:1007E400938E938C0101409181BE04D040A101D02D
:0607F40001D0FAD712004B
:1007FA0001016F6B706B72DC03C168F104C169F1AE
:10080A00F40E01016A6F000E6B6F1EDE00C003F169
:10081A0001C004F140DE01016F6B010E706F5EDCF6
:10082A0003C168F104C169F1C20E01016A6F000EC9
:10083A006B6F0ADE00C003F101C004F12CDE010176
:10084A006F6B020E706F4ADC03C168F104C169F173
:10085A00850E01016A6F000E6B6FF6DD00C003F1B1
:10086A0001C004F118DE01016F6B030E706F36DCF4
:10087A0003C168F104C169F1760E01016A6F000EC5
:10088A006B6FE2DD00C003F101C004F104DE010177
:10089A006F6B040E706F22DC03C168F104C169F149
:1008AA00B30E01016A6F000E6B6FCEDD00C003F15B
:1008BA0001C004F1F0DD01016F6B050E706F0EDCF3
:1008CA0003C168F104C169F1050E01016A6F010EE5
:1008DA006B6FBADD00C003F101C004F1DCDD120068
:1008EA000101666B676B800E6719006E800E005CF3
:1008FA0002E1050E665D36E203C168F104C169F1E1
:10090A00140E6A6F010E6B6F9FDD020E0325E16EF6
:10091A00000E0421E26E300E6625006E00C0E6FF6E
:10092A0066C168F1C8DC00C055F101C056F100C0CB
:10093A0068F101C069F119C16AF11AC16BF150DCA1
:10094A0003C168F104C169F119C16AF11AC16BF1F5
:10095A004BDDA1DD2C0E01016F6F0EDC0101664B30
:06096A00672BC1D712004B
:100970002FDCD00E0101686FDADC880E686FD7DCDF
:04098000BDDC1200C8
:1009840000C015F09EA017D001013E4B3F2B850EF1
:10099400CF6EED0ECE6E9E90000E006E3F51005C49
:1009A40002E13E51090806E2454B462B3E6B3F6B84
:0C09B400010E4F6F9E9015C000F0110066
:1009C00060EC09F06F6A6E6AFF0E936EF18EFF0E97
:1009D0008A6EFF0E806E010E926E810EC26E8E0EBA
:1009E000C16E946A010ED56E0A0EAF6EAC84CEDE77
:1009F000F2DD0050010A03E1F3DD00C057F1070EFC
:100A00000101546FDFDD03C168F104C169F1580EC3
:100A100001016A6F000E6B6F1CDD00C003F101C0A5
:100A200004F13EDD51C068F152C069F13F0E010191
:100A30006A6F000E6B6F0DDD00C051F001C052F007
:100A400000C06FF101C070F156EC00F000C062F11F
:100A500001C063F1606B616B6351615D02E16251E2
:100A6000605D0FE260C166F160515124E96E615131
:100A70005220EA6EEECF67F1BCDD0101604B612BC5
:100A8000EBD7606B616B000E615D02E1110E605D82
:100A900017E260C166F1C7DD00C05EF1000E5F6F56
:100AA000A30E0C6E550E0D6E0D2EFED70C2EFCD720
:100AB0005EC16FF1C1EC00F00101604B612BE3D727
:100AC00081DD0101546BB7DD01016F6B706B73EC5D
:100AD00000F0010E0101546F90DE0101546B8DDEB8
:100AE000330E0B6EBB0E0C6EDF0E0D6E0D2EFED791
:100AF0000C2EFCD70B2EFAD700000000010E0101CE
:100B0000546F60DD010E0101546F3C6B800E3C1987
:100B1000006E800E040A005C43E23CC100F0000E4F
:100B20003CBFFF0E016E0036009001361C0E002403
:100B3000646F010E0120656F3CC100F0000E3CBFE8
:100B4000FF0E016ED60E046E060E056EF7DD0D0E5D
:100B50000026020E012264C1E1FF65C1E2FF00C070
:100B6000E6FF01C0E6FF3CC100F0000E3CBFFF0EF7
:100B7000016E0036009001361C0E0024E96E010E55
:100B80000120EA6EEECF68F1EECF69F103C16AF1A0
:100B900004C16BF1F5EC00F083DC01013C2BB6D70E
:100BA00011DD01013C6B576B5C6B5D6B546B3EEC74
:100BB00001F018DE300ECD6ECD80ED0ECF6E850EBD
:100BC000CE6E9E90F29C9D90F29E010E0101546F9C
:100BD0005C6B5D6B03C168F104C169F1300E6A6F33
:100BE000000E6B6F36DC00C003F101C004F158DC6D
:100BF0000101596B080E5B6F5A6B880E586F880E97
:100C0000686F000E696F03C16AF104C16BF1F5EC06
:100C100000F05E6B5F6B000E5F5D02E1050E5E5DD6
:100C200016E25E510325E96E5F510421EA6EEECFB4
:100C300001F00150200A08E15E510325E16E5F5189
:100C40000421E26E300EE66E5E4B5F2BE4D728DCAB
:100C5000B9DC8EDE1A0E0B6E5E0E0C6E6E0E0D6E15
:100C60000D2EFED70C2EFCD70B2EFAD70000020E4D
:100C700001011B6F576B3C6BAEDC0050010A2EE18B
:100C8000AFDC00C057F116D001011B7127D01B73D8
:100C900025D01B7523D0030E5A5D01E25A2B1ED0BE
:100CA0005A51000801E25A0719D08CDCA6DD8ADC13
:100CB00015D014D001015751310AE6E05751320ADC
:100CC000E6E05751330AE5E057512B0AE4E057516B
:100CD0002D0AE6E057511B0AE8E0EBD701015C4B17
:100CE0005D2B010E546F1BA14BD003C168F104C1F1
:100CF00069F1160E6A6F000E6B6F29EC02F000C0EE
:100D000003F101C004F15CC168F15DC169F119C171
:100D10006AF11AC16BF1F5EC00F05E6B5F6B000ECF
:100D20005F5D02E1050E5E5D16E25E511925E96E1A
:100D30005F511A21EA6EEECF01F00150200A08E15E
:100D40005E511925E16E5F511A21E26E300EE66E9A
:100D50005E4B5F2BE4D703C168F104C169F119C18F
:100D60006AF11AC16BF1F9EC01F000C003F101C0A6
:100D700004F150EC02F0090E01016F6FC1EC00F0BC
:100D800001011BA301D0B1DD090E6F6FC1EC00F0B2
:100D900001016F6B706B73EC00F001013C6B0CD0C8
:100DA000200E596F16D0400E596F13D0600E596F38
:100DB00010D0596B0ED00DD03C51000AF1E03C51DF
:100DC000010AF1E03C51020AF1E03C51030AF1E072
:100DD000F2D7020E0B6E040E0C6EBA0E0D6E0D2EB7
:100DE000FED70C2EFCD70B2EFAD700001BA514D073
:100DF0003CC100F0000E3CBFFF0E016E00360090BB
:100E000001361C0E0024E96E010E0120EA6EEECFC1
:100E100055F1EECF56F105D057DC00C055F101C0B9
:100E200056F155C168F156C169F103C16AF104C1B7
:100E30006BF1F5EC00F05E6B5F6B000E5F5D02E145
:100E4000050E5E5D16E25E510325E96E5F510421D9
:100E5000EA6EEECF01F00150200A08E15E51032551
:100E6000E16E5F510421E26E300EE66E5E4B5F2B49
:100E7000E4D7010E546F50EC02F0800E01013C19D2
:100E8000006E800E030A005C04E22C0E6F6FC1EC52
:100E900000F00101546B6F6B706B73EC00F003C1D9
:100EA00068F104C169F1210E01016A6F000E6B6FD8
:100EB00029EC02F000C003F101C004F150EC02F093
:100EC00001016F6B010E706F73EC00F003C168F1EC
:100ED00004C169F11A0E01016A6F000E6B6F29ECF3
:100EE00002F000C003F101C004F15AC168F1000E24
:100EF000696F19C16AF11AC16BF1F5EC00F003C119
:100F000068F104C169F119C16AF11AC16BF1F9EC18
:100F100001F000C003F101C004F150EC02F0010146
:100F20006F6B020E3C25706F73EC00F003C168F12B
:100F300004C169F1530E01016A6F000E6B6F29EC59
:100F400002F000C003F101C004F1020E0024E16EC2
:100F5000000E0120E26E310E3C25006E00C0E6FF5F
:100F600050EC02F01C0E01016F6F020E3C25706FF9
:100F700073EC00F055C168F156C169F103C16AF123
:100F800004C16BF1F5EC00F050EC02F0010E010130
:100F9000546F3C2B800E3C19006E800E040A005CDE
:100FA000D8A0FDD62C0E6F6FC1EC00F05AC168F1CD
:100FB000000E0101696F03C16AF104C16BF1F5EC28
:100FC00000F050EC02F08A72010E0101546F070E1E
:0A0FD0001B17E2EC02F050D6FFD729
:1012C00010EE16F0050E006E020E016EBA0EF66EEE
:0E12D000110EF76E000EF86E5CEC03F01200CB
:100FDA00000000000000005F000000070007001486
:100FEA007F147F14242A7F2A122313086462364945
:100FFA005522500005030000001C22410000412236
:10100A001C0014083E081408083E08080050300066
:10101A0000080808080800606000002010080402A0
:10102A003E5149453E00427F4000426151494621B6
:10103A0041454B311814127F1027454545393C4A22
:10104A004949300171090503364949493606494972
:10105A00291E0036360000005636000008142241C8
:10106A000014141414140041221408020151090630
:10107A00324979413E7E1111117E7F494949363EF6
:10108A00414141227F4141221C7F494949417F090F
:10109A000909013E4149497A7F0808087F00417FD2
:1010AA0041002040413F017F081422417F404040D7
:1010BA00407F020C027F7F0408107F3E4141413E7F
:1010CA007F090909063E4151215E7F0919294646D1
:1010DA004949493101017F01013F4040403F1F20FA
:1010EA0040201F3F4038403F6314081463070870CC
:1010FA0008076151494543007F4141000204081035
:10110A00200041417F000402010204404040404067
:10111A00000102040020545454787F48444438386B
:10112A0044444420384444487F3854545418087E70
:10113A000901020C5252523E7F0804047800447D91
:10114A0040002040443D007F1028440000417F4079
:10115A00007C041804787C08040478384444443831
:10116A007C14141408081414187C7C080404084815
:10117A0054545420043F4440203C4040207C1C20CE
:10118A0040201C3C4030403C44281028440C50501D
:10119A00503C4464544C44000836410000007F002F
:1011AA0000004136080010080810087846414678C1
:0411BA004E623D0044
:0711BE004761696E3D20004E
:0F11C5004D4350333432342032382F303820002D
:0F11D400436F6E666967204144433138623D00C6
:1011E3007061756C666A756A6F40667265652E66B6
:0211F300720088
:0211F500D10027
:0511F70043482E3D00FD
:1011FC00204D435033343234204144432031382085
:0E120C00626974732032382F30382F31300071
:0F121A00332E53696D756C20313862202020000F
:0F122900322E4C65637420414443313062200003
:101238003132333435363738393031323334353664
:0F124800373839303132333435363738393000B2
:0F1257002B2E204741494E2055502020202000AB
:0F126600312E4E756D6572205472616D652000DA
:101275007061756C666A756A6F40667265652E6623
:021285007200F5
:101287003132333435363738393031323334353615
:011297000056
:0F1298002D2D455343203D204D454E5520200020
:0212A7009400B1
:0F12A9002D2E204741494E20444F574E20200004
:0512B8004348303D0039
:0212BD00E3004C
:020000040030CA
:0D000100220F0EFFFF80FF0FC00FE00F4029
:00000001FF
